:1000000012038C7409120398744D120398744112F0
:10001000039874541203987443120398744812039B
:10002000987420120398744712039874411203982D
:10003000744D1203987445120398740A120398744D
:100040000D120398741A900404F07420120398742B
:100050006E1203987475120398746D12039874628B
:100060001203987465120398747212039874201224
:100070000398746F12039874661203987420120325
:1000800098746D1203987461120398747412039833
:100090007463120398746812039874651203987459
:1000A0007312039874201203987472120398746583
:1000B000120398746D120398746112039874691294
:1000C0000398746E1203987469120398746E120385
:1000D000987467120398743A120398742012039864
:1000E000900404E0900403F01202DD7420120398DF
:1000F0007465120398746E120398747412039874E2
:100100006512039874721203987420120398743164
:10011000120398742D1203987434120398743A12CF
:1001200003987420120398120280900403E0900454
:1001300002F0900402E0C0E07404C0E0D0F0D0E02F
:10014000C395F0600DA2D292F765F054807003025F
:1001500000EB900402E0C0E07401C0E0D0F0D0E019
:10016000C395F0A2D292F765F0548060030200EBD1
:10017000900404E0C0E0900402E0C0E0D0F0D0E0E1
:10018000C395F0900404F0900404E0C0E07400C053
:10019000E0D0F0D0E095F07003020228900404E073
:1001A000C0E07400C0E0D0F0D0E0C395F0A2D292DD
:1001B000F765F054806003020228742012039874DB
:1001C000491203987427120398746C120398746C84
:1001D00012039874201203987474120398746112B5
:1001E0000398746B1203987465120398743A12039F
:1001F0009874201203987405C0E0900402E0C0E0F7
:10020000D0F0D0E0C395F0900403F0900404E0C077
:10021000E0900403E0C0E0D0F0D0E0C395F090049B
:1002200004F01202DD02004A742012039874531283
:100230000398746F12039874721203987472120305
:1002400098747912039874201203987479120398A1
:10025000746F1203987475120398742012039874C3
:100260006C120398746F1203987473120398746578
:10027000120398740A120398740D12039802000373
:100280007400900403F01203A0900401F0900401A4
:10029000E0120398900401E0C0E0740DC0E0D0F0DB
:1002A000D0E095F070030202D2900403E0C0E07445
:1002B0000AD0F0A4C0E0900401E0C0E07430C0E0D7
:1002C000D0F0D0E0C395F0D0F025F0900403F00218
:1002D0000286740A120398740D1203982274009017
:1002E0000400F07402C0E07402C0E0900400E0C0BA
:1002F000E0900403E0C0E0740AC0E0D0F0D0E084F5
:10030000C0F07430D0F025F0D082D083F090040398
:10031000E0C0E0740AC0E0D0F0D0E084900403F0C4
:10032000900400E004F0D0F0C395F0600AA2D292ED
:10033000F765F054806005C0F00202E77400900495
:1003400000F07402C0E07402C0E07402C0E09004E7
:1003500000E0C0E0D0F0D0E0C395F0C0E0D082D0A3
:1003600083E0120398900400E004F0D0F0C395F00D
:10037000600AA2D292F765F054806005C0F00203D3
:1003800046740A120398740D1203982275985275D8
:100390008920758DFDD28E223099FDC299F5992262
:0803A0003098FDC298E5992296
:00000001FF
